:100000000C941E060C9404280C9431280C9446067B
:100010000C9446060C9446060C9446060C94460630
:100020000C9446060C9446060C9415130C94460644
:100030000C9446060C9446060C9446060C94460610
:100040000C945E280C9446060C944C2C0C948F2C2B
:100050000C9446060C9446060C9446060C944606F0
:100060000C9446060C9446067918DB18BA18BD188D
:10007000C018C318C618C918CC18DB18D5180D1A23
:100080000F1A0F1A0D1A0F1A0F1A0F1A0F1A0F1A2A
:100090000F1A0F1A0F1A0F1A0F1A0F1A0F1A0F1A18
:1000A00093190F1A0F1A0F1A0F1A0F1A04190F1A91
:1000B0000F1A0F1A0F1A0F1A0F1A0F1A0F1A0F1AF8
:1000C0000F1A0F1A0F1A0F1A0F1A0F1A9F199F19CA
:1000D0009F199F199F199F199F199F199F190F1AEF
:1000E0000F1A0F1A0F1A0F1A0F1A04199E199E19B8
:1000F0009E199E190F1AAC19B219B819BE19C41954
:10010000CA19D019D619E019EA19F419FE194519B6
:1001100007190F1A0F1A0F1A0F1A93190F1A0F1A1D
:100120000F1A0F1A0F1A0F1A0F1A0F1A9D199D196D
:100130009D199D190F1AAC19B219B819BE19C41915
:10014000CA19D019D619E019EA19F419FE19451976
:1001500007190F1A0F1A0F1A0F1A9319421A421A77
:10016000421A421A421A421A421A421A421A421AAF
:10017000421A421A421A591B591B591B591B591B27
:10018000591B871A911A9B1AA51A031B0D1B1C1BBE
:100190002D1BB51CCA1CD61CDF1CEE1C131D1C1D00
:1001A000651D2E1D77207D2083208A209820BA206F
:1001B000D820456E746572206D656E752E2E2E00EA
:1001C000546F67676C6564206D6963726F50504D42
:1001D00000546F67676C656420696E76657274653C
:1001E000642050504D2100546F67676C6564205443
:1001F00058206D7574696E672100546F67676C6570
:10020000642074656C656D65747279210050726F3D
:10021000746F636F6C206572726F72207769746897
:100220002052580054696D656F7574207768656E4B
:1002300020636F6E6E656374696E6720746F205201
:100240005800507265737320616E79206B65792058
:10025000746F2063616E63656C00436F6E6E6563DF
:1002600074696E6720746F2052582C20706F776508
:100270007220757020746865205258202877697440
:10028000682062696E6420706C7567206966206EF4
:100290006F74207573696E6720616C776179732064
:1002A00062696E642900546F67676C656420276912
:1002B0006D6D656469617465206F75747075742700
:1002C00000546F67676C65642027736C61766520E6
:1002D0006D6F64652700546F67676C6564202761E4
:1002E0006C776179732062696E642700546F676769
:1002F0006C65642050504D206368616E6E656C20A3
:100300006C696D69740053657420525353492069B8
:100310006E6A656374696F6E206368616E6E656C8A
:100320002028303D3D64697361626C652900536526
:10033000742050504D206D696E696D756D20737914
:100340006E630053657420626561636F6E20696E31
:1003500074657276616C0053657420626561636FC9
:100360006E2064656C617900536574206265616319
:100370006F6E206672657175656E637920696E2097
:10038000487A3A20303D64697361626C652C205074
:10039000783D504D52206368616E6E656C20782CFC
:1003A0002046783D465253206368616E6E656C202E
:1003B00078005365742050574D2073746F7020641B
:1003C000656C61792028302064697361626C6564B2
:1003D0002C20312D323535203D3D20302E317320FB
:1003E0002D2035306D696E29005365742050504DB5
:1003F0002073746F702064656C61792028302064EC
:10040000697361626C65642C20312D323535203D75
:100410003D20302E3173202D2035306D696E29003E
:10042000536574206661696C736166652064656CF0
:1004300061792028302064697361626C65642C20C6
:10044000312D323535203D3D20302E3173202D2089
:1004500035306D696E29002A2A2A2A2A2A2A2A2A50
:100460002A2A2A2A2A2A2A2A2A2A2A2A2A2A2A2AEC
:100470002A2A2A2A0052582041636B6564202D20C5
:1004800072657665727420737563636573736675E0
:100490006C21002A2A2A2A2A2A2A2A2A2A2A2A2AAD
:1004A0002A2A2A2A2A2A2A2A2A2A2A2A2A2A2A2AAC
:1004B000002A2A2A2A2A2A2A2A2A2A2A2A2A2A2AC6
:1004C0002A2A2A2A2A2A2A2A2A2A2A2A2A2A00528E
:1004D000582041636B6564202D20757064617465DC
:1004E000207375636365737366756C21002A2A2A0D
:1004F0002A2A2A2A2A2A2A2A2A2A2A2A2A2A2A2A5C
:100500002A2A2A2A2A2A2A2A2A2A0056616C696457
:100510002063686F69636573206172653A205B319F
:100520005D2D5B31365D20286368616E6E656C20E1
:10053000312D31362900536574206F7574707574D0
:1005400020666F7220706F727420005B585D2061AE
:10055000626F7274206368616E67657320616E6498
:10056000206578697420525820636F6E6669670051
:100570005B535D20736176652073657474696E6783
:100580007320746F205258005B525D20726576654F
:1005900072742052582073657474696E6773207486
:1005A0006F2064656661756C747300557365206EA9
:1005B000756D62657273205B312D445D20746F2010
:1005C0006564697420706F727473205B452D515D92
:1005D00020666F722073657474696E677300202DD6
:1005E00020726563656976657220636F6E66696700
:1005F000757261746F722C20727820737720000AF4
:100600000A6F70656E4C52536E67200053657420FC
:1006100073657269616C2062617564726174653AB8
:10062000200056616C69642063686F696365733A82
:100630002031202D20342B34202F2032202D203823
:10064000202F2033202D20382B34202F2034202D14
:10065000203132202F2035202D2031322B34202FF5
:100660002036202D20313600536574204368616E9A
:100670006E656C20636F6E6669673A20005365741F
:100680002044617461726174652028302D32293AEA
:10069000200053657420486F70206368616E6E653A
:1006A0006C7320286D61782032342C207365706162
:1006B000726174656420627920636F6D6D61732966
:1006C0002076616C69642076616C75657320312DCC
:1006D0003235353A2000536574206368616E6E656B
:1006E0006C2073706163696E6720287831306B48C5
:1006F0007A293A200053657420524620706F77653E
:10070000722028302D37293A200053657420524634
:10071000206D6167696320286865782920652E67E8
:100720002E20307844454144463030443A2000532E
:1007300065742062617365206672657175656E63AC
:10074000792028696E20487A293A20005B5A5D207A
:10075000656E746572207265636569766572206383
:100760006F6E66696775726174696F6E2075746902
:100770006C79005B465D20646973706C61792061FF
:10078000637475616C206672657175656E63696509
:10079000732075736564005B525D2063616C6375E3
:1007A0006C6174652072616E646F6D206B65792079
:1007B000616E6420686F70206C697374005B495DC2
:1007C000207265696E697469616C697A6520736508
:1007D0007474696E677320746F20736B65746368DB
:1007E0002064656661756C7473005B585D2072658A
:1007F00076657274206368616E67657320616E64EC
:100800002065786974206D656E75005B535D20739B
:100810006176652073657474696E677320746F20E8
:10082000454550524F4D20616E64206578697420B3
:100830006D656E7500557365206E756D62657273BA
:10084000205B302D395D20746F20656469742070E1
:100850006172616D657465727300202D2053797328
:1008600074656D20636F6E66696775726174696F18
:100870006E000A0A6F70656E4C52536E672000510D
:1008800029204F7574707574206265666F726520DB
:100890006C696E6B20283D465329203A2000502970
:1008A00020536C617665206D6F64652028657870D3
:1008B0006572696D656E74616C293A20004F29205C
:1008C00054696D65642042494E44206174207374FC
:1008D000617274757020203A20004E292050504DCE
:1008E000206F7574707574206C696D69746564200F
:1008F000202020203A200044495341424C454400E6
:100900004D292050504D205253534920746F20637D
:1009100068616E6E656C202020203A20004C2920F2
:1009200050504D206D696E696D756D2073796E63E1
:10093000202875732920203A200044495341424C15
:100940004544004B29204661696C736166652062ED
:100950006561636F6E20696E74762E2028312D32AA
:10096000353573293A20004A29204661696C736144
:10097000666520626561636F6E2064656C617920D5
:1009800028302D323535203D3E20313073202D204A
:100990003135306D696E293A200049292046616958
:1009A0006C7361666520626561636F6E206672714B
:1009B0002E203A200048292050574D2073746F7024
:1009C0002064656C6179202020202020203A2000BE
:1009D00047292050504D2073746F702064656C61FE
:1009E00079202020202020203A200046292046611E
:1009F000696C736166652064656C617920202020D4
:100A00002020203A200050574D206368616E6E65AB
:100A10006C200066756E6374696F6E3A2000292041
:100A2000706F72742000506F776572546F776572C3
:100A300000445446205548462033322D62697420C4
:100A400031306368004F70656E4C52536E67525878
:100A5000206D696E6920342F36636800466C7974A6
:100A6000726F6E2F4F72616E6765525820554846FF
:100A70002038636800525820747970653A20004429
:100A8000697361626C656400487A00203D3D200016
:100A900043616C63756C61746564207061636B6540
:100AA0007420696E74657276616C3A200042292068
:100AB0004D6963726F202868616C66292050504D23
:100AC000202020203A00412920496E766572746505
:100AD000642050504D20696E20202020203A0030A4
:100AE00029204D7574652062757A7A657220286DAB
:100AF0006F73746C79293A003929205365726961E2
:100B00006C2062617564726174653A00736D617224
:100B100074506F7274004672536B79005472616E38
:100B200073706172656E740044697361626C6564B0
:100B30000038292054656C656D657472793A2020FF
:100B40002020202020003729204368616E6E656CCC
:100B500020636F6E6669673A202000362920446161
:100B60007461726174652028302D32293A2020206A
:100B700000352920486F70206368616E6E656C7364
:100B80003A2020202020003429204368616E6E65C1
:100B90006C2073706163696E673A202000332920EE
:100BA000524620706F7765722028302D37293A2001
:100BB0002020003229205246206D616769633A2067
:100BC0002020202020202020003129204261736530
:100BD000206672657175656E63793A202020000089
:100BE00000000700020100000304060000000000EE
:100BF00000000001020408102040800102040810D7
:100C00002001020408102004040404040404040263
:100C10000202020202030303030303000000002395
:100C2000002600290000000000250028002B0000FD
:100C3000000000240027002A00007D2D11241FBE83
:100C4000CFEFD8E0DEBFCDBF13E0A0E0B1E0E8E039
:100C5000F1E602C005900D92A83CB107D9F716E065
:100C6000A8ECB3E001C01D92AE38B107E1F71CE07B
:100C7000CCE3DCE004C02297FE010E94862ECA333A
:100C8000D107C9F70E94B92D0C9482300C94000052
:100C900080917305813019F482E08093730580910F
:100CA0007305833019F484E0809373050895A89543
:100CB0000895DC01ED91FC910190F081E02D099502
:100CC00008952091740530917505382748E0C901D1
:100CD000880F991F37FF06C09C0151E2252750E17C
:100CE000352701C09C01415091F730937505209341
:100CF0007405089588E38093760580E092ECA1E086
:100D0000B0E08093770590937805A0937905B09330
:100D10007A0587E08093830580EC92E9ADEEB9E136
:100D200080937B0590937C05A0937D05B0937E0511
:100D300085E0809384058DEE9EEFADEABEED809355
:100D40007F0590938005A0938105B0938205E5E827
:100D5000F5E080E090E0863028F4DC01AE54BC4F32
:100D60002C9101C020E0219301968831910599F7DB
:100D700082E080939D058AE080939E05089580EC33
:100D800091EDA8E9BBE18093BB059093BC05A093CE
:100D9000BD05B093BE0580E090E0A0E0B0E5809393
:100DA000BF059093C005A093C105B093C205E3ECC5
:100DB000F5E080E081938F5F8031E1F70895A0E056
:100DC000B0E0E5EEF6E00C944F2ED82F0E94B42848
:100DD0006115710581059105C9F30E94F22E1092EB
:100DE0007F05109280051092810510928205C4E063
:100DF000812C912C54018A94C0907F05D09080055D
:100E0000E0908105F0908205FE2CED2CDC2CCC24AA
:100E10000E94ED2EA50194010E942E2E6C0D7D1DC9
:100E20008E1D9F1D60937F057093800580938105C3
:100E300090938205C15001F7DD2309F450C005E805
:100E400015E0E801A12CB12C62E3C62ED12CE12CD7
:100E5000F12C8881882309F442C0B39419F40E94CC
:100E60007A063DC00E94ED2EA70196010E942E2E0B
:100E7000E1E0E60FA5E8B5E08A2F801B8A1520F493
:100E80008D918E13F9CFE9CF2091840530E0A0E158
:100E9000B7E20E94C62D9B01AC01AE2FB0E00E94CC
:100EA000D52D40907B0550907C0560907D0570901D
:100EB0007E05640D751D861D971D4090BB055090E5
:100EC000BC056090BD057090BE05461657066806C5
:100ED000790618F2E993A39488E1A812BACFCDB7A6
:100EE000DEB7E0E10C946B2E8436910520F4BC0152
:100EF00080E090E017C09C018E3B910528F42A55B4
:100F00003109AAE0B0E00CC0823D910528F4245BD1
:100F10003109A4E6B0E004C02D5C3109A8E5B2E0D7
:100F20000E94C62DA4E6B0E09B01AC010E94D52D25
:100F3000089590E08C599F4F0E947407089561E0D6
:100F400086E00E94612960E086E00E949A2982E0A2
:100F50008093B00085E08093B10061E083E00E945F
:100F6000612960E083E00E949A290895CF93DF937E
:100F7000EC010097E9F061E086E00E949A299E0169
:100F800040E050E068E478EE81E090E00E942E2E90
:100F90002F3F31054105510529F020F02FEF30E0BA
:100FA00040E050E02093B3008091B000806107C022
:100FB00060E086E00E949A298091B0008F7E809345
:100FC000B000DF91CF91089560E08EE00E9461292A
:100FD00061E08FE00E94612961E080E10E94612967
:100FE00060E082E00E94612961E084E00E94612962
:100FF000089542E050E068E476E080E00E94E42753
:101000000895E3E0F0E089E080935700E491E67012
:1010100081E0E63009F080E00895CF93DF93C82F98
:101020000E940108882381F0DFB781E08093720578
:10103000F8940E94570688E180936000C093600096
:10104000C1110E945706DFBFDF91CF9108958F92A3
:101050009F92AF92BF92CF92DF92EF92FF92CF9387
:10106000FC01C0A5EC2FE770F0E0E658FC4FA08132
:10107000B0E0C7FF03C024E130E002C02FE030E061
:10108000FC0197A183E1989FF0011124E25CFE4FDF
:1010900080809180A280B380A20FB31F20E43FE143
:1010A0004DE750E00E94E02DA50194010E940C2E16
:1010B0008C2F887149F469017A01E0EDCE0EE7E0EA
:1010C000DE1EE11CF11C1BC0C7FF05C060E47AE80E
:1010D0008CE29EE004C060E07EEE8AEB9BE069015A
:1010E0007A01F8EBCF0EFBE0DF1EE11CF11CA5013D
:1010F00094010E940C2EC20ED31EE41EF51EC701E1
:10110000B60169517C4F8F4F9F4F28EE33E040E08E
:1011100050E00E940C2EA8EEB3E00E94D52DCF9196
:10112000FF90EF90DF90CF90BF90AF909F908F9007
:1011300008958F3F910551F048F0811522E0920704
:1011400038F08115934030F482E0089580E00895EE
:1011500081E0089583E00895A0E0B0E0E2EBF8E0DC
:101160000C94582EEB018A01B82FB695A0E0288187
:101170003981F80120832A813B8121832C813D81A3
:1011800022832E813F812383688179814A815B811B
:101190002C813D81EE81FF819F2F9295990F990FB0
:1011A000907C272F2370922B252F2370220F220F44
:1011B000922B232F23702295207F922BF80194836A
:1011C0000B5F1F4F2896AF5FBA1788F680FF24C0C9
:1011D000888199810E949908D82E8A819B810E94DA
:1011E0009908E82E8C819D810E949908F82E8E81A5
:1011F0009F810E949908F0E4DF9EA001112490E1F4
:10120000E99E90011124242B282BE4E0FE9EB001DE
:101210001124262BF8012083CDB7DEB7E7E00C942C
:10122000742E803223E0920708F1883E23E0920773
:1012300040F48F519340E4E096958795EA95E1F765
:101240000895803D27E0920718F48C5D934008953F
:10125000883928E0920768F4885C974074E0969596
:1012600087957A95E1F78D509C4F089580E090E046
:1012700008958FEF93E008958C30910540F4A4E039
:10128000880F991FAA95E1F7885D9C4F0895843FC8
:1012900023E0920718F484529C4F0895811524E0AE
:1012A000920740F48657934FF4E0880F991FFA9500
:1012B000E1F7089580E998E008959C013695279517
:1012C00025753575821B930B9C012373337396959B
:1012D00087959695879583739373820F931F9C01CF
:1012E00054E0369527955A95E1F7280F391F2F704E
:1012F0003F7041E051E0249FC001259F900D349F35
:10130000900D1124892F08954298882319F0000028
:10131000419A02C0000041980000429A00000895DE
:10132000429A000086B14298000081700895CF93E0
:10133000DF93D82F5C9A42985C98C8E08D2F807814
:101340000E948409DD0FC150C9F74298DF91CF9107
:1013500008958F770E9497090895CF93DF93D82F30
:10136000C8E08D2F80780E948409DD0FC150C9F735
:101370004298DF91CF910895CF93DF934298C8E0D0
:1013800080E0D82FDD0F0E9490098D0FC150C9F762
:10139000DF91CF9108950E94A9090E94BC095C9A2F
:1013A0000895A1E0B0E0E7EDF9E00C945D2E8068CF
:1013B00069830E9497096981862F0E94AD095C9A12
:1013C0002196E2E00C94792ECF93C0917F05C82737
:1013D000E82FF0E0EA58FA4F678589E70E94D109C3
:1013E0006C2F8DE30E94D1096C2F82E40E94D109F9
:1013F000CF91089586E20E94CB090895CF93DF93A1
:10140000EC016C818CE10E94D1096D818DE10E941B
:10141000D1096E818EE10E94D1096F8180E20E9424
:10142000D109688581E20E94D109698582E20E9422
:10143000D1096A8583E20E94D1096B8584E20E940A
:10144000D1096C8585E20E94D1096D858AE20E94EE
:10145000D1096E858EE60E94D1096F858FE60E94C4
:10146000D109688980E70E94D109698981E70E94D2
:10147000D1096A8982E70E94D109DF91CF9108954D
:10148000CF92DF92EF92FF92CF93DF936B017C01BB
:10149000C11488E3D8068CE9E8068CE1F80628F543
:1014A000C701B60120E836E948E950E00E940C2E59
:1014B000E901689760E879E687E69FEF0E94E82DEA
:1014C0006C0D7D1D8E1D9F1DF2E0660F771F881F1E
:1014D000991FFA95D1F721E732E040E050E00E94F1
:1014E0000C2EF22EE32E80E421C0C701B60120E0CD
:1014F0003DE241E351E00E940C2EE901689760E073
:1015000073ED8EEC9EEF0E94E82D6C0D7D1D8E1DFF
:101510009F1D660F771F881F991F21E732E040E06B
:1015200050E00E940C2EF22EE32E80E66C2F6F719D
:10153000680F85E70E94D1096E2D86E70E94D109C8
:101540006F2D87E70E94D109DF91CF91FF90EF9037
:10155000DF90CF900895682F8DE60E94D1090895FD
:101560008F929F92AF92BF92CF92DF92EF92FF92B3
:10157000CF93DF93D82F83E00E94CB09809371052E
:1015800084E00E94CB098093700560E086E00E94B1
:10159000D10961E087E00E94D1096FE789E00E94EC
:1015A000D10965E08AE00E94D10962E18BE00E94E6
:1015B000D10965E18CE00E94D1096DEF8DE00E94B8
:1015C000D10960E08EE00E94D109DD2319F08BE2A1
:1015D00091E008C020919D0533E1239FC0011124B3
:1015E000825C9E4F0E94FE096CE880E30E94D10954
:1015F0006FE082E30E94D10962E483E30E94D10993
:1016000080919E0587FF02C064E101C06AE084E327
:101610000E94D1096AE285E30E94D1096DE286E366
:101620000E94D10964ED87E30E94D10960E088E35C
:101630000E94D10960E089E30E94D109D11109C05B
:10164000C0907F05D0908005E0908105F0908205E4
:1016500007C0C5E9CC2EC1ECDC2EED2CCEEDFC2E66
:10166000CAE38F2C9924AA24BB24682D8C2F0E94B6
:10167000D109682D85E08C0F0E94D109FE2CED2C3C
:10168000DC2CCC24CF5FCE3361F76FEF83E40E9474
:10169000D1096FEF84E40E94D1096FEF85E40E94C5
:1016A000D1096FEF86E40E94D109DD2311F066E0D5
:1016B00002C0609183058DE60E94D10960E089E750
:1016C0000E94D109609184058AE70E94D10960E0F7
:1016D00083E70E94D10960E084E70E94D109D1111B
:1016E00009C060917B0570917C0580917D0590918A
:1016F0007E0504C060EC72E98DEE99E10E94400A1B
:10170000DF91CF91FF90EF90DF90CF90BF90AF909F
:101710009F908F90089561E087E00E94D10964E274
:101720008EE70E94D10963E088E00E94D10960E061
:1017300088E00E94D10965E087E00E94D10962E05B
:1017400085E00E94D10983E00E94CB098093710556
:1017500084E00E94CB0980937005089583E00E9485
:10176000CB098093710584E00E94CB0980937005BA
:1017700061E087E00E94D1096AE070E080E090E0DB
:101780000E94D7280E948B0B00000895CF92DF9211
:10179000FF920F931F93CF93DF931F92CDB7DEB7C6
:1017A000082F162F8EE399830E94D109F02EC02EA8
:1017B0009981D92E8C2D8F19811738F4F6016191FA
:1017C0006F018FE70E94D109F5CF64E085E00E94A8
:1017D000D10983E00E94CB098093710584E00E94C7
:1017E000CB09809370050E94B42860936C057093B8
:1017F0006D0580936E0590936F0569E087E00E9408
:10180000D10981E0809373050F90DF91CF911F91F3
:101810000F91FF90DF90CF9008950F931F930E9438
:10182000C60B80917305813099F40E94B428009111
:101830006C0510916D0520916E0530916F05601B50
:10184000710B820B930B603A76488140910548F307
:1018500080917305813031F46EE971E082EE95E09C
:101860000E94A02A1F910F9108950F931F938091BA
:101870007305823021F41092730581E020C08091BD
:1018800073058130D9F40E94B42800916C05109141
:101890006D0520916E0530916F05601B710B820BF9
:1018A000930B613A76488140910540F061E087E012
:1018B0000E94D1091092730582E001C080E01F915F
:1018C0000F910895CF93DF93EC014AE050E06D2F24
:1018D00070E082EE95E00E946E2B6EE282EE95E063
:1018E0000E94722ABE0184E0769567958A95E1F799
:1018F0006F7077274AE050E082EE95E00E946E2BF1
:10190000DF91CF910895D82FC0E0CD1790F4439A7E
:10191000299A64E670E080E090E00E94D72843981E
:10192000299864E670E080E090E00E94D728CF5FBD
:10193000ECCF6CE271E080E090E00E94D728E4CF29
:101940000F931F93CF93DF93EC01062F15E01150F7
:1019500051F0CE010E946930081741F0602FCE018E
:101960000E947130F4CF82E00E94830CDF91CF910E
:101970001F910F910895A0E0B0E0E1ECFCE00C9421
:101980004F2E482E562EC0E0D0E0612C712CE12C59
:10199000F12C00E010E041100CC06090D40586E40A
:1019A000689E3001112459E1E52EF12C0AEB15E077
:1019B0001EC091E049120FC06090D405E6E46E9E0F
:1019C00030011124FBE16F0E711C49E2E42EF12C71
:1019D00006E715E00CC082E0481209C028E1622E3B
:1019E00077247394EE24E394F12C03ED15E0430186
:1019F0008C0E9D1E10927505109274053401A62C54
:101A0000A818B12CC30101966C01AE14BF04A8F450
:101A1000A00EB11E511006C0C3010E946930F5012D
:101A2000808305C0F5016081C3010E94A00CF5010F
:101A300080810E9461063601E2CFC301511018C0B7
:101A4000C3010E946930B82EC6010E9469302B2D57
:101A500030E0322F2227282B809174059091750554
:101A60008217930779F4C0E0D0E05524539493CFC4
:101A70003601609175050E94A00C60917405C60145
:101A80000E94A00CC05EDE4FC13E92E0D90708F470
:101A900082CF852DCDB7DEB7E0E10C946B2E61E0EF
:101AA00082E00E94BB0C089560E082E00E94BB0CC3
:101AB0008091D305853028F084E08093D3050E947F
:101AC0004F0D8091D3058093D405089561E080E0A7
:101AD0000E94BB0C61E081E00E94BB0C089560E0B5
:101AE00080E00E94BB0C882351F060E081E00E94FE
:101AF000BB0C882321F080917605883349F00E9441
:101B0000BF060E947A0681E00E94DF060E94660DF1
:101B10000895882319F06AEA71E002C06EEA71E064
:101B200082EE95E00E94A02A0895FF920F931F93E2
:101B3000CF93DF9369EC7BE082EE95E00E944C2A24
:101B400040917B0550917C0560917D0570917E05EB
:101B50002AE030E082EE95E00E94752B63EB7BE09B
:101B600082EE95E00E944C2A40917F0550918005BD
:101B7000609181057091820520E130E082EE95E070
:101B80000E94752B6DE97BE082EE95E00E944C2A65
:101B90004AE050E06091830582EE95E00E949D2B23
:101BA00067E87BE082EE95E00E944C2A4AE050E034
:101BB0006091840582EE95E00E949D2B61E77BE0B9
:101BC00082EE95E00E944C2AC5E8D5E0F12C8E010A
:101BD00088818823A9F0FF2031F061EB71E082EE6B
:101BE00095E00E946F2A21964AE050E0F80160815A
:101BF00082EE95E00E94662BF394F8E1FF12E7CFA6
:101C000082EE95E00E947A2A6BE57BE082EE95E019
:101C10000E944C2A4AE050E060919D0582EE95E0DA
:101C20000E949D2B66E47BE082EE95E00E944C2AA8
:101C3000E0919E05E770F0E0EE0FFF1FEE57FC4FBE
:101C40006081718182EE95E00E94A02A61E37BE0D1
:101C500082EE95E00E944C2A80919E058871883022
:101C600069F028F4811113C068E27BE00CC0803178
:101C700041F0883161F46CE07BE005C06CE17BE011
:101C800002C066E17BE082EE95E00E948E2A68EF5A
:101C90007AE082EE95E00E944C2A409177055091BF
:101CA00078056091790570917A052AE030E082EE3E
:101CB00095E00E94752B6FED7AE082EE95E00E9430
:101CC0004C2A8091BF0580710E94890D66EC7AE0F4
:101CD00082EE95E00E944C2A8091BF0580740E949C
:101CE000890D6DEA7AE082EE95E00E944C2A80919F
:101CF000BF0580720E94890D60E97AE082EE95E06E
:101D00000E944C2A86E795E00E942708AB01BC019F
:101D10002AE030E082EE95E00E94572B6BE87AE0F3
:101D200082EE95E00E944C2A86E795E00E94270803
:101D30009B01AC0160E472E48FE090E00E940C2E05
:101D4000BA01A9012AE030E082EE95E00E94572B0B
:101D500068E87AE082EE95E00E948E2ACDB7DEB781
:101D6000E5E00C94762E8F929F92AF92BF92CF9225
:101D7000DF92EF92FF92811107C06FE77AE082EE67
:101D800095E00E948E2A2FC090E00E94740724E6FE
:101D900030E040E050E00E940C2ECA01B9012AE078
:101DA00030E040E050E00E940C2E49015A016B01E6
:101DB0007C012AE030E0B501A40182EE95E00E94AA
:101DC000572B6EE282EE95E00E94722A2AE030E004
:101DD000B701A60182EE95E00E94572B63E782EEE1
:101DE00095E00E94B22AFF90EF90DF90CF90BF90D5
:101DF000AF909F908F9008951F93CF93DF9365E7E7
:101E00007AE082EE95E00E944C2A80919F05813015
:101E100041F46CE57AE082EE95E00E948E2A10E0B3
:101E200050C0823019F465E47AE0F5CF843019F4BB
:101E300061E37AE0F0CF853091F766E27AE0EBCFAC
:101E4000C12FD0E0C930D1050CF441C068E3610F67
:101E500082EE95E00E94722A6EE17AE082EE95E0D1
:101E60000E944C2ABE016F5F7F4F4AE050E082EE35
:101E700095E00E94362B63E17AE082EE95E00E94C5
:101E80004C2AC156DA4FE981E03218F566E07AE073
:101E900082EE95E00E944C2A8981803130F06DE617
:101EA00073E082EE95E00E946F2A69816F7070E0A6
:101EB0006F5F7F4F4AE050E082EE95E00E943F2B3B
:101EC0001F5F80914805181708F4BACF0FC061E36F
:101ED000BECFEF70F0E0EE0FFF1FEE56FC4F6081BB
:101EE000718182EE95E00E94A02AEACF6BEE79E044
:101EF00082EE95E00E944C2A8091B7050E94B30EB5
:101F000060ED79E082EE95E00E944C2A8091B80560
:101F10000E94B30E65EB79E082EE95E00E944C2AB8
:101F20008091B9050E94B30E6AE979E082EE95E0EE
:101F30000E944C2A4091AF055091B0056091B105C7
:101F40007091B205411551056105710539F12AE01D
:101F500030E082EE95E00E94752B67E679E082EE34
:101F600095E00E944C2A8091B3050E949907AB012D
:101F7000BC012AE030E082EE95E00E94752B63E41C
:101F800079E082EE95E00E944C2A4AE050E06091B0
:101F9000B40582EE95E00E949D2B06C06AE379E0CD
:101FA00082EE95E00E948E2A6DE179E082EE95E066
:101FB0000E944C2A6091B5057091B6054AE050E048
:101FC00082EE95E00E94872B60E079E082EE95E05A
:101FD0000E944C2A6091AE05603450F470E06F5F4F
:101FE0007F4F4AE050E082EE95E00E943F2B06C012
:101FF00067EF78E082EE95E00E948E2A6AED78E045
:1020000082EE95E00E944C2A8091AD0580FF03C0CE
:1020100063EB71E002C067EB71E082EE95E00E9435
:10202000A02A6DEB78E082EE95E00E944C2A809128
:10203000AD0582700E94890D6EE978E082EE95E030
:102040000E944C2A8091AD0584700E94890D6FE733
:1020500078E082EE95E00E944C2A8091AD05887070
:102060000E94890DDF91CF911F9108950F931F93C7
:10207000CF93DF93209145052F3FA9F56FEF75E0D2
:1020800082EE95E00E944C2A80E893E00E94620C68
:102090006EED75E082EE95E00E944C2A8091460537
:1020A000909147050E94620C6BEA75E082EE95E024
:1020B0000E948E2A68E875E082EE95E00E948E2AE2
:1020C00060E775E082EE95E00E948E2A6BE475E091
:1020D00082EE95E00E948E2A82EE95E00E947A2A96
:1020E0000E94FC0E68C012160CF065C0332727FD55
:1020F00030958091480590E0821793070CF45BC0FF
:1021000066E375E082EE95E00E944C2A60914505F9
:10211000772767FD70954AE050E082EE95E00E94D7
:102120003F2B6BE075E082EE95E00E944C2A10E0B8
:1021300008E2809149051817D0F5C12FD0E0CC0FE7
:10214000DD1FC65BDA4F288130E080914505992775
:1021500087FD909501972817390739F56BEB71E0EA
:1021600082EE95E00E946F2A4AE050E0602F82EEF6
:1021700095E00E94662B6FEB71E082EE95E00E9485
:102180006F2AE981EF70F0E0EE0FFF1FEE56FC4F73
:102190006081718182EE95E00E946F2A63EC71E0AC
:1021A00082EE95E00E946F2A0F5F1F5FC2CF82EE22
:1021B00095E00E947A2ADF91CF911F910F910895A7
:1021C000FF920F931F93CF93DF93C5E8D5E0F12CD7
:1021D0008E0188818823D1F165EC71E082EE95E073
:1021E0000E946F2A4AE050E06F2D82EE95E00E9437
:1021F000662B62ED71E082EE95E00E946F2A2196D7
:10220000F801208130E0A0E1B7E20E94C62D9B01D9
:10221000AC01A0918405B0E00E94D52DAB01BC01BA
:1022200080917B0590917C05A0917D05B0917E0504
:10223000480F591F6A1F7B1F2AE030E082EE95E0AD
:102240000E94752BF394F8E1FF12C2CFCDB7DEB731
:10225000E5E00C94762E1092DF0485E6E0EEF4E0E3
:10226000DF011D928A95E9F70895CF93C82F8F3724
:1022700019F0883009F045C0E091DF04EE23D9F170
:10228000E150E093DF04F0E0E052FB4F10826DE09C
:1022900070E082EE95E00E945906C0E08091DF0474
:1022A000C81760F4EC2FF0E0E052FB4F608170E063
:1022B00082EE95E00E945906CF5FF0CF60E270E0B9
:1022C00082EE95E00E9459066DE070E082EE95E0A6
:1022D0000E945906C0E08091DF04C81778F5EC2F02
:1022E000F0E0E052FB4F608170E082EE95E00E94EA
:1022F0005906CF5FF0CF67E082EE95E00E94722A28
:102300001DC08B3119F40E942B111AC08D30C1F001
:102310008A30B1F08091DF04843668F76C2F70E06A
:1023200082EE95E00E945906E091DF0481E08E0F75
:102330008093DF04F0E0E052FB4FC08380E001C0F7
:1023400081E0CF910895CF93C82F0E94B428609365
:10235000C8047093C9048093CA049093CB04C093BB
:10236000DD04CC2329F040E051EE60E070E004C0D1
:1023700040E855E260E070E082EE95E00E94FC2CBF
:10238000CF9108959091CC04492F4F7050E0BA013D
:102390006F5F7F4F292F30E0E4E035952795EA9570
:1023A000E1F76217730759F0FA01E353FB4F80839B
:1023B00081E0890F8F70907F892B8093CC040895E2
:1023C0006EE770E082EE95E00E9459060895A3E161
:1023D000B1E0EDEEF1E10C94502EE5E8F5E0712C62
:1023E0008191882321F0739428E17212F9CF66ED70
:1023F00071E082EE95E00E94A02A4AE050E0672D4D
:1024000082EE95E00E949D2B80E00E94B00A0E941F
:102410008B0B8E010E5F1F4FC12CD12C7601C39404
:1024200066246A945C2C0E94A8284B015C012091D0
:10243000840530E0A0E1B7E20E94C62D9B01AC010B
:10244000C701B6010E94E82D20917B0530917C05E3
:1024500040917D0550917E05620F731F841F951F6B
:102460002091BB053091BC054091BD055091BE0542
:10247000261737074807590718F4F80160822AC061
:102480008C2D0E94E40961E070E080E090E00E9401
:10249000D728F80110820E94A828681979098A09AA
:1024A0009B09643F71408105910540F40E94FA093F
:1024B000F8019081981778F78083EDCF85B150FEB1
:1024C00005C08B7D85B9439A299A04C0846285B979
:1024D000439829982FEFC21AD20AE20AF20A0F5F34
:1024E0001F4F8FEFC816D104E104F10409F09ACF11
:1024F000CE019395FC01D82E7FEF68EC2E2F281B80
:10250000271510F051E056C0DE01129651E02FEF72
:1025100041E03D91321710F0322F01C0452F5F5F2F
:102520005F3F11F0232FF5CF4193242F30E0A1E03E
:10253000B0E0AC0FBD1FA20FB31F5C93413079F028
:10254000DE01A20FB31F5C93423049F0AFEFBFEF43
:10255000AC0FBD1FA20FB31F6C934E3F78F6A2E0E5
:10256000B0E0AC0FBD1FA20FB31F7C934D3F30F600
:10257000A3E0B0E0AC0FBD1FA20FB31F6C93BECFA2
:10258000452F242F30E0FC01E20FF31F6081AFEFF5
:10259000B0E0AC0FBD1FA20FB31F2C91621748F41F
:1025A0004150DC01A40FB11D2C9120836C9341118B
:1025B000E8CF5F5F571520F3372D369520E02317BE
:1025C00070F4DC01A20FB11D4C91522F530FFC018E
:1025D000E50FF11D50815C9340832E5FF0CFF5E84D
:1025E000EF2EF5E0FF2E8C01802F8D19871598F4C2
:1025F000F801C1908F014AE050E06C2D82EE95E029
:102600000E94662B6CE282EE95E00E94722AF7012E
:10261000C1927F01E9CF82EE95E00E947A2A81E0A3
:10262000CD5EDE4FEFE00C946C2E1F920F920FB632
:102630000F9211241F932F933F934F935F936F93A8
:102640007F938F939F93AF93BF93CF93DF93EF933A
:10265000FF93C0918600D09187008091870490916C
:1026600088042091A904211155C09E01281B390B13
:102670008091BF059091C005A091C105B091C205A0
:1026800085FD02C036952795253C49E03407B8F111
:1026900040910A0150E060E070E02CE1B695A7950A
:1026A000979587952A95D1F70097A105B10521F453
:1026B00081E090E0A0E0B0E084179507A607B70797
:1026C000D8F480910A018F3FB9F040E080910A016F
:1026D000481780F4842F90E0880F991FFC01E7577A
:1026E000FB4F20813181FC01E55FFE4F3183208368
:1026F0004F5FECCF1092AA0410920A010BC02D3B41
:1027000082E0380720F080910A018031D8F08FEF05
:1027100080930A01D0938804C0938704FF91EF91BE
:10272000DF91CF91BF91AF919F918F917F916F91E9
:102730005F914F913F912F911F910F900FBE0F907E
:102740001F90189510910A0181E0810F80930A0172
:10275000C9010E941109E12FF0E0EE0FFF1FE757BA
:10276000FB4F91838083D6CF83E0809380008AE9FA
:10277000809381008091BF0586FD05C08091810016
:102780008064809381008FEF9FEF90938900809306
:10279000880080916F00806280936F0008950E948E
:1027A000540D8091D405843011F41092D40508950D
:1027B0006F3018F086958058089589E0689F802DC5
:1027C00011240895A0E0B0E0E8EEF3E10C94572E58
:1027D000C82F0E94B4280091380410913904209128
:1027E0003A0430913B046B017C01C01AD10AE20A21
:1027F000F30A9701860149E8C41643E1D406E104CF
:10280000F10410F010923C04609338047093390482
:1028100080933A0490933B042091A9048FEF820F98
:102820008230D8F5E0913C04EE2309F44EC1E1304A
:1028300011F482E0B8C1E03108F034C181E08E0FBC
:1028400080933C04F0E0E757FB4FC083803109F0F0
:10285000ACC1EBE8F4E0213029F4A181A695A6955E
:10286000808108C080819181A92FA695A695A69503
:1028700096958795A03148F4B0E090E0AA0FBB1F71
:10288000A55FBE4F11969C938E931092AA04329628
:1028900084E0E939F807F9F688C1233009F005C169
:1028A000E0913C04E11104C0CF3009F07EC10DC1BC
:1028B000E83148F481E08E0F80933C04F0E0E85763
:1028C000FB4FC08372C1E83109F0ECC0C111EAC00E
:1028D00040E050E0ABE0CA01B3E0880F991FBA9521
:1028E000E1F7A49F9001A59F300D1124F901E7574E
:1028F000FB4F6081E1817E2F777075956795FC01B4
:10290000EE0FFF1FE55FFE4F71836083F901E6570D
:10291000FB4FB081B695B695B695E181FE2FF29545
:10292000FF0FF07E6F2F6B2BE695E695E6957E2FD9
:10293000777075956795FC01EE0FFF1FE35FFE4F03
:1029400071836083F901E557FB4FB081B295B6956D
:10295000B695B370C181DC2FDD0FDD0F6D2F6B2BB2
:10296000C295C695C695C370E281E170EE0FEE0F79
:102970007E2F7C2B75956795FC01EE0FFF1FE15FA5
:10298000FE4F71836083F901E357FB4FB081B69529
:10299000E181FE2FF795FF27F7956F2F6B2BE695BB
:1029A0007E2F777075956795FC01EE0FFF1FEF5E28
:1029B000FE4F71836083F901E257FB4FB081B295FE
:1029C000BF70E181FE2FF295F07F6F2F6B2BE295A8
:1029D000EF707E2F777075956795FC01EE0FFF1FE6
:1029E000ED5EFE4F71836083F901E157FB4FB081CB
:1029F000BB1FBB27BB1FC181DC2FDD0F6D2F6B2BD6
:102A0000CC1FCC27CC1FE281E370EE0F7E2F7C2BF6
:102A100075956795FC01EE0FFF1FEB5EFE4F71830E
:102A20006083F901EF56FB4FB081B695B695E18111
:102A3000FE2FF295FF0FFF0FF07C6F2F6B2BE695AB
:102A4000E6957E2F777075956795FC01EE0FFF1F59
:102A5000E95EFE4F71836083F901EE56FB4F2081E2
:102A60002295269527703181E32FEE0FEE0FEE0FA2
:102A70006E2F622B732F729576957770759567958B
:102A8000FC01EE0FFF1FE75EFE4F718360834F5F17
:102A90005F4F4230510509F01ECF80919F0483FFA4
:102AA0001092AA0410923C0480C0243009F07DC02A
:102AB00060913C0461110BC0C83AB1F410927505E5
:102AC0001092740588EA0E94610681E06CC0613052
:102AD00019F4C093370404C0623031F4C093360453
:102AE0008C2F0E9461065AC0E09136042E2F30E0F0
:102AF000220F331F462F50E0C90102968417950715
:102B00003CF0633268F7FA01EA57FB4FC083E8CF25
:102B10002D5F3F4F8C2F90E060917405709175058B
:102B20004217530749F4982F8827862797279093B1
:102B300075058093740532C06817790769F580912F
:102B40003704813049F5E13118F080E18093360493
:102B5000F0903604CAE8D4E000E010E00F15D0F49D
:102B6000FE013197808190E0982F88272881822B61
:102B700063E0969587956A95E1F70E941109F8013F
:102B8000EE0FFF1FE55FFE4F918380830F5F1F4FA6
:102B90002296E4CF1092AA0410923C0480913C0447
:102BA000882319F08F5F80933C04CDB7DEB7E8E04F
:102BB0000C94732EE82FF0E0E654FA4FE185E031F3
:102BC00050F4F894F0E0EE0FFF1FE55FFE4F8081B8
:102BD000918178940895E03121F0E13131F483E17D
:102BE00001C082E10E94F629089580E092E00895F4
:102BF000A2E2B0E0EEEFF5E10C944D2E9E012F5FC6
:102C00003F4F80E1D9011D928A95E9F764E072E0B7
:102C100082EE95E029A33AA30E94A02A0E94AE0B5F
:102C20001D8A1E8A1F8A188E312C212C00E0812CCF
:102C3000912C540170E4472E71EE572E7DE9672EDA
:102C400078E1772EE0E5CE2EE3ECDE2EE12CF12CC0
:102C500084EF91E0A0E0B0E08D8F9E8FAF8FB8A39E
:102C600080EC91EDA8E9BBE1898F9A8FAB8FBC8F87
:102C700080E491EEADE9B8E1898B9A8BAB8BBC8B8C
:102C800082EE95E00E94B42B892B09F4E1C082EE1C
:102C900095E00E94E12B9C0133272C32310509F489
:102CA00042C0ACF42332310509F0ABC019821A825C
:102CB0001B821C821D821E821F82188619861A861C
:102CC0001B861C861D861E861F86188A60C02434BB
:102CD000310529F02335310509F4B2C092C064E40E
:102CE00082EE95E00E94722A2AE030E040E451EE44
:102CF0006DE978E182EE95E00E94002B6CE282EEB5
:102D000095E00E94722A2AE030E040EC51ED68E93B
:102D10007BE182EE95E00E94002B6CE282EE95E072
:102D20000E94B22AADCF0F5F043009F0A9CF2981EC
:102D30003A814B815C81A8EEB3E00E94D52D698B6E
:102D40007A8B8B8B9C8B2D813E814F8158850E9485
:102D5000D52D698F7A8F8B8F9C8F29853A854B85EE
:102D60005C852D8F3E8F4F8F58A32D853E854F85D7
:102D700058890E94D52D6B017C0160323EE47307B7
:102D80008105910530F462E38CE10E94D10900E0F5
:102D900077CF603345E774078105910510F462E24F
:102DA000F3CF60345CE975078105910510F466E2A4
:102DB000EBCF80E5C81683ECD806E104F10410F4EB
:102DC00062E1E2CF90E6C9169AEED906E104F10479
:102DD00010F465E1D9CFA0E7CA16A1E1DA06A1E0B7
:102DE000EA06F10410F461E0CFCFB0EACB16B6E802
:102DF000DB06B1E0EB06F10410F463E0C5CF65E05B
:102E0000C3CF10ED180F1A3008F03ACFE1E0F0E030
:102E1000EC0FFD1F24E0029FE00DF11D1124208125
:102E2000318142815381AAE0B0E00E94D52D610F2B
:102E3000711D811D911D608371838283938320CFD7
:102E400049885A886B887C88812C912C540118CF32
:102E500081149104A104B10489F4C301B2010E9458
:102E6000400A61E070E080E090E00E94D7281D8A6F
:102E70001E8A1F8A188E312C22242A948D8D9E8DB5
:102E8000AF8DB8A188169906AA06BB06D0F40E9499
:102E9000FA092D893E894F89588D280F311D411D12
:102EA000511D2D8B3E8B4F8B588F381608F4382EC2
:102EB000821508F4282E3FEF831A930AA30AB30A57
:102EC00056C0C301B20128EE33E040E050E00E945A
:102ED0000C2EBA01A9012AE030E082EE95E00E94B2
:102EE000572B6CE282EE95E00E94722A4AE050E095
:102EF000632D82EE95E00E94662B6CE282EE95E0F7
:102F00000E94722A6D897E898F89988DA50194010E
:102F10000E940C2EBA01A9012AE030E082EE95E071
:102F20000E94572B6CE282EE95E00E94722A4AE0E2
:102F300050E0622D82EE95E00E94662B6CE282EEFC
:102F400095E00E94B22A4C0C5D1C6E1C7F1C898D82
:102F50009A8DAB8DBC8D84159505A605B70520F41B
:102F600049885A886B887C88812C912C5401298946
:102F70003A894B895C89283E33404105510509F067
:102F80007FCEA296E2E10C94692EACE1B0E0EBECCE
:102F9000F7E10C94572E0E94B4286B017C0181E06C
:102FA0000E94B00A14E703E0198361E0CE010196A4
:102FB0000E940D0C009373050E948B0B6AEF70E06A
:102FC00080E090E00E94D72880917305833089F4D7
:102FD00082EE95E00E94B42B892B59F40E94B4280C
:102FE0006C197D098E099F096038734C894C91409A
:102FF000D8F280917305833009F44FC08FE70E94A7
:10300000A9090E94BC098983843511F083E05CC062
:103010000E94BC0910924605809347050E94BC0996
:103020002091460530914705280F311D3093470503
:10303000209346050E94BC09809348050E94BC0964
:1030400080934905813110F7F12C0F2D10E080910C
:10305000490590E0880F991F0817190740F40E944E
:10306000BC09F801E65BFA4F8083F394EECF80E76A
:10307000898361E0CE0101960E940D0C83E080936C
:1030800073050E948B0B62E370E080E090E00E9489
:10309000D72880917305833011F482E015C08FE743
:1030A0000E94A9090E94BC098983803509F0AECF2E
:1030B0000FE915E00E94BC09F80181938F01F5E04A
:1030C0000A3B1F07B9F781E06C96E8E00C94732E79
:1030D00080914505992787FD9095A92FB92FFC016F
:1030E0003196EB30F10508F066C0EC5CFF4F0C94B4
:1030F000842E62E778E082EE95E00E948E2A80E8D6
:1031000093E00E94620C6AE578E082EE95E00E940E
:103110008E2A65E378E082EE95E00E948E2A6BE0CD
:1031200078E082EE95E00E948E2A6AEE77E082EEE9
:1031300095E00E948E2A6DEB77E082EE95E00E948A
:103140008E2A67E977E082EE95E00E948E2A63E797
:1031500077E082EE95E00E948E2A6CE477E082EEC2
:1031600095E00E948E2A82EE95E00E947A2A0E94C3
:10317000950D21C06FE277E01AC06AE077E017C0D2
:1031800065EF76E014C066ED76E011C062E976E0A6
:103190000EC06DE776E00BC068E676E082EE95E063
:1031A0000E948E2A62E276E002C06CE076E082EE57
:1031B00095E00E948E2A6AE070E080E090E00E9434
:1031C000D72882EE95E00E94B42B892B29F082EE5D
:1031D00095E00E94E12BF5CF0895ACE1B0E0E3EF7C
:1031E000F8E10C94572E909145059F3F09F023C1BB
:1031F000482F50E0FA013A97EF36F10508F00FC179
:10320000E15CFF4F0C94842E61E172E0A0C06DE19F
:1032100072E082EE95E00E94A02A85E789838BE127
:10322000EFE9F5E0DE01129601900D928A95E1F743
:103230006CE1CE0101960E940D0C0E948B0B83E085
:103240008093730568EC70E080E090E00E94D728DE
:1032500080917305843009F0E2C08FE70E94A909CC
:103260000E94BC098983853509F0D9C06DEE74E0F0
:1032700082EE95E00E948E2A6FEC74E082EE95E07B
:103280000E948E2A61EB74E096C065E372E082EEE4
:1032900095E00E94A02A89E6898361E0CE0101962B
:1032A0000E940D0C0E948B0B83E08093730568ECE9
:1032B00070E080E090E00E94D72880917305843010
:1032C00009F0ADC08FE70E94A9090E94BC0989835B
:1032D0008E010E5F1F4F7E014DE1E40EF11C0E9436
:1032E000BC09F80181938F01EE15FF05C1F78BE151
:1032F000FE013296AFE9B5E001900D928A95E1F7B3
:103300008981893409F08BC063E974E082EE95E02D
:103310000E948E2A65E774E082EE95E00E948E2A74
:1033200067E574E048C06FE472E082EE95E00E94C9
:10333000A02A8EEF8093450572C08052875080533B
:1033400090914805981708F066C06EE572E082EE2D
:1033500095E00E94A02A63C084E18093450560E265
:1033600074E029C085E18093450569EE73E023C0D0
:1033700086E18093450562EB73E01DC087E1809391
:10338000450568E673E017C088E18093450567E569
:1033900073E011C089E18093450563E473E00BC0DD
:1033A0008AE1809345056EE273E005C08BE180936E
:1033B000450566E073E082EE95E00E948E2A2FC0FC
:1033C0006CEE72E082EE95E00E948E2A8091AD054F
:1033D00091E01DC066ED72E082EE95E00E948E2ABB
:1033E0008091AD0592E013C061EC72E082EE95E051
:1033F0000E948E2A8091AD0594E009C066EA72E0D1
:1034000082EE95E00E948E2A8091AD0598E0892792
:103410008093AD058FEF809345050E94361082EEB4
:1034200095E00E94B42B892B09F45BC182EE95E0F4
:103430000E94E12BF4CF0E943511882309F451C179
:103440008091DF04811104C08FEF8093450541C155
:1034500040E050E060E070E080EE94E00E94FB2EDF
:1034600040914505042F112707FD1095212F312F7D
:10347000F8013197EB31F10508F01BC1E255FF4F20
:103480000C94842E552747FD50952091480530E037
:10349000241735070CF40DC18B019C010150110953
:1034A00021093109003211052105310558F0C0907C
:1034B0004905EBE4F5E0F12CD12CA8E2EA2E4150CD
:1034C00051090FC0FA01E156FA4F61506083D9C02B
:1034D000DF0111972C9130E02417350729F0F39480
:1034E0003296FC10F5CFCBC00E2D10E020E030E07E
:1034F000061717072807390741F42081DA01A1567A
:10350000BA4F11962C93DD24D394E394E8CF6F3F08
:1035100071058105910511F008F0CBC06093B705E6
:10352000B0C06F3F71058105910511F008F0C1C071
:103530006093B805A6C06F3F71058105910511F034
:1035400008F0B7C06093B9059CC02091E0042062E8
:103550002037E9F440E050E060E070E081EE94E074
:103560000E94FB2E9B01AC01DC01CB010197A1095C
:10357000B1090897A105B10508F0AEC0A4EDB0E30C
:103580000E94D52D6A5E7C4A8A46954E24C0263616
:10359000E9F440E050E060E070E081EE94E00E94E9
:1035A000FB2E9B01AC01DC01CB010197A109B10904
:1035B0000797A105B10508F08FC0A8EAB1E60E94FF
:1035C000D52D645E7C438E46944E05C06115710511
:1035D0008105910579F08B019C010054114E2D4914
:1035E00038410138F0EF1F07FAEF2F07F2E03F07ED
:1035F00008F05FC06093AF057093B0058093B1058C
:103600009093B2053EC06F3F71058105910511F0A1
:1036100008F04FC06093B30534C08B019C0101508A
:103620001109210931090F3F11052105310508F064
:1036300040C06093B40525C08B019C01045C194017
:10364000210931090D344DE114072105310528F414
:103650007093B6056093B50514C0611571058105B9
:10366000910521F48FEF8093AE050BC06134710595
:1036700081059105F0F461506093AE0502C0DD2034
:10368000C1F08091DE0481111AC080917F05909174
:103690008005A0918105B09182050196A11DB11D03
:1036A00080937F0590938005A0938105B093820558
:1036B00006C060E772E082EE95E00E94A02A0E94B8
:1036C0002B118FEF809345056AE082EE95E00E9412
:1036D000B22A0E94361005C061E070E080E090E000
:1036E0007ACF6C96E8E00C94732E6AE572E082EE75
:1036F00095E00E948E2A62E472E082EE95E00E94DC
:103700008E2A82EE95E00E94B42B892B31F082EE56
:1037100095E00E94E12B0E94ED180E94C5178230AF
:1037200029F0833051F46DE072E002C064E272E08F
:1037300082EE95E00E948E2A08958FEF80934505D2
:103740001092DE040E943610809145058E3F69F08C
:1037500082EE95E00E94B42B892BB1F382EE95E0C6
:103760000E94E12B0E94ED18EFCF08950F931F9355
:10377000109145051F3F09F0D2C0893409F457C0A4
:1037800000F5883309F469C058F4803309F477C030
:1037900008F061C08B3109F440C08132B1F1B9C089
:1037A000813409F487C030F4893309F466C0803469
:1037B00061F1AFC0823409F48EC0863409F448C088
:1037C000A8C0823609F487C078F4883531F128F42E
:1037D0008235C1F18335E1F09CC08A3509F494C08B
:1037E000813609F467C095C0823761F128F48636C6
:1037F00079F18936E1F08DC0883779F08A3709F49C
:1038000083C0833709F085C003C061E172E015C051
:103810000E94660D6EE872E004C00E946F0D68EAB7
:1038200072E082EE95E00E94A02A8EEF70C00E94A6
:103830007A060E94BF0667EC72E082EE95E00E9475
:10384000A02A67C081E00E94DF0660EE72E0F5CF3B
:103850000E94E0105EC080535AC06AEF71E082EEB1
:1038600095E00E948E2A90919E0588E0890F8871CC
:10387000977E892B80939E051AC089E048C067EE29
:1038800071E082EE95E00E948E2A8091BF059091B2
:10389000C005A091C105B091C20520E182278093A7
:1038A000BF059093C005A093C105B093C2051093C6
:1038B00045052FC061ED71E082EE95E00E948E2AF1
:1038C0008091BF059091C005A091C105B091C2053E
:1038D00040E4842710C060EC71E082EE95E00E9425
:1038E0008E2A8091BF059091C005A091C105B0912D
:1038F000C20520E282278093BF059093C005A09364
:10390000C105B093C20502C00E94751B8FEF809362
:103910004505809145058E3F09F0D4C0DDC00E9469
:103920003511882309F4D8C08091DF04811104C0C7
:103930008FEF80934505C6C040E050E060E070E046
:1039400080EE94E00E94FB2E00914505112707FDB3
:103950001095212F312FF8013197E930F10508F04A
:10396000B4C0E753FF4F0C94842E8B019C0101548B
:10397000114E2D4938410F37104F2A4F324008F071
:10398000A4C060937B0570937C0580937D05909324
:103990007E0577C060937F057093800580938105D5
:1039A0009093820581E08093DE046BC068307105DE
:1039B0008105910508F089C06093830562C08B0181
:1039C0009C0101501109210931090A301105210515
:1039D000310508F07AC06093840553C061EB71E053
:1039E00080EE94E00E94353010E0009799F00E943C
:1039F0000F30009779F0183130F4E12FF0E0EA58F9
:103A0000FA4F87871F5F61EB71E080E090E00E94D2
:103A10003530EBCF1831A8F5E12FF0E0EA58FA4F36
:103A200017861F5FF7CF653071058105910508F096
:103A30004CC060939D0525C08B019C01015011096C
:103A4000210931090630110521053105F0F52091D4
:103A50009E05287F262B20939E0513C08B019C0179
:103A600001501109210931090115124C214031057C
:103A700060F560937705709378058093790590934E
:103A80007A058091DE04811113C080917F059091A9
:103A90008005A0918105B09182050196A11DB11DFF
:103AA00080937F0590938005A0938105B093820554
:103AB0000E942B118FEF809345056AE082EE95E01E
:103AC0000E94B22A0E94681807C060E772E082EE86
:103AD00095E00E94A02AECCF1F910F9108958FEFDF
:103AE000809345051092DE040E9468188091450578
:103AF0008E3F69F082EE95E00E94B42B892BB1F3E2
:103B000082EE95E00E94E12B0E94B61BEFCF6AE0A7
:103B100070E080E090E00E94D72882EE95E00E945D
:103B2000B42B892B29F082EE95E00E94E12BF5CF92
:103B30000895CF93C82F682F82EE95E00E940E2C37
:103B400090916A059C2790936A05CF910895A1E012
:103B5000B0E0EDEAFDE10C945D2E99830E94991D81
:103B60009981892F0E94991D2196E2E00C94792E6B
:103B70001F93CF93DF93182FEB0110926A0565EB2B
:103B800070E082EE95E00E94590662E670E082EEF7
:103B900095E00E945906812F0E94991DCE010E9436
:103BA000A71DDF91CF911F91089560916A0582EE64
:103BB00095E00E940E2C0895A1E2B0E0E2EEFDE156
:103BC0000C94592E7B018A018C3009F452C108F003
:103BD00040C0863009F4BCC018F5833009F491C0A8
:103BE00070F4813009F472C0823009F047C26BE191
:103BF00070E082E00E94B81D0FE915E078C08430C3
:103C000009F487C0853009F039C26091490570E038
:103C1000660F771F85E00E94B81D0AE415E086C094
:103C2000893009F4A7C070F4873009F49BC088304C
:103C300009F024C261E070E088E00E94B81D809124
:103C4000D40522C28A3009F4CAC08B3009F4F1C00D
:103C500015C28A3609F474C1D8F4873609F439C11B
:103C600038F4853609F40DC1863609F41EC106C242
:103C7000883609F436C1893609F000C261E070E087
:103C800089E60E94B81D0E947A060E94BF06F4C110
:103C90008D3609F4D3C138F48B3609F490C18C36D3
:103CA00009F499C1EBC18E3609F4DBC1873C09F0F8
:103CB000E5C161E070E087EC0E94B81D81E00E94E0
:103CC000991D0E94D51D10926B05E2C169E270E05A
:103CD00081E00E94B81D06E715E0F80181918F018F
:103CE0000E94991DF5E00F391F07B9F7CFC1F80100
:103CF00081918F010E94991DF5E00A3B1F07B9F7DA
:103D0000C5C161E070E083E00E94B81D0E94C51744
:103D1000BBC161E070E084E00E94B81D81E00E94B8
:103D2000991D0E94D51D0E94F815B2C180914905C8
:103D300090E0880F991F98012A54354028173907B9
:103D400008F0A4C1F80181918F010E94991DEECF66
:103D500062E070E086E00E94B81D80E893E00E9477
:103D6000A71D94C161E070E087E00E94B81D8091BA
:103D700048058AC186E6898361E0CE0101960E94EA
:103D80000D0C0E948B0B83E08093730568EC70E050
:103D900080E090E00E94D728809173058430D9F4A8
:103DA0008FE70E94A9090E94BC098983863469F4BF
:103DB00060E270E089E00E94B81D10E20E94BC0938
:103DC0000E94991D1150D1F761C161E070E089E056
:103DD0000E94B81D51C161E070E089E052C169E103
:103DE00070E08AE00E94B81D1092BA052091720519
:103DF0008091BF059091C005A091C105B091C20509
:103E0000222311F0806801C08F778093BF059093C3
:103E1000C005A093C105B093C2050AEB15E0F801F7
:103E200081918F010E94991DF5E0033D1F07B9F7AD
:103E30002DC161E270E08BE00E94B81D8091AA0460
:103E40008F3F39F08091AA0491E0980F9093AA04D3
:103E500002C08091AA040E94991D10E0812F0E9447
:103E6000DA150E943C090E94A71D1F5F1031B1F7AF
:103E70000DC161E070E08CE00E94B81D8091D30517
:103E800003C161E070E085E60E94B81D89E2E81692
:103E9000F10409F0F8C0D801E6E7F5E08D918193CF
:103EA00085E0EF39F807D1F7E7C061E070E086E61A
:103EB0000E94B81DEBE1EE16F10409F0E4C0D80150
:103EC000EFE9F5E08D91819385E0EA3BF807D1F7C2
:103ED000D3C061E070E087E60E94B81D0E94660DC5
:103EE000CBC061E070E088E60E94B81D85E7898359
:103EF0008BE1EFE9F5E0DE01129601900D928A95D3
:103F0000E1F76CE1CE0101960E940D0C0E948B0B33
:103F100083E08093730560E273E080E090E00E94AC
:103F2000D72880917305843009F0ADC08FE70E94D7
:103F3000A9090E94BC098983853509F0A4C09CC0E9
:103F400061E070E08AE60E94B81D89E6898361E03D
:103F5000CE0101960E940D0C0E948B0B83E0809392
:103F6000730560E273E080E090E00E94D7288091C2
:103F70007305843009F087C08FE70E94A9090E9469
:103F8000BC0989838E010E5F1F4F7E01EDE1EE0EAD
:103F9000F11C0E94BC09F80181938F01EE15FF0509
:103FA000C1F78BE1FE013296AFE9B5E001900D92C9
:103FB0008A95E1F78981893409F065C05DC061E0C7
:103FC00070E08BE60E94B81DF80180818093D405D3
:103FD0000E946F0D51C061E070E08CE60E94B81D38
:103FE000F0E2EF16F10461F487E6898380E2F801DC
:103FF000DE01129601900D928A95E1F761E203C00D
:1040000087E4898361E0CE0101960E940D0C0E9435
:104010008B0B83E0809373056CE474E080E090E0A8
:104020000E94D72880917305843069F58FE70E943C
:10403000A9090E94BC09873431F51EC061E070E017
:104040008DE60E94B81D89E1E816F104E1F4D8017B
:10405000EAEBF5E08D91819385E0E33DF807D1F738
:104060000BC061E070E08EE60E94B81DF80180810F
:104070008093D3050E944F0D81E006C061E070E09F
:104080008AEC0E94B81D80E00E94991D0E94D51DF7
:10409000A196E6E00C94752EA0E0B0E0E2E5F0E237
:1040A0000C94572ECAECD3E014E606E035E0F32E6C
:1040B00044E0E42E53E0D52E62E0C62E82EE95E079
:1040C0000E94B42B892B09F49BC082EE95E00E94DC
:1040D000E12B282F809335044091340450E0473081
:1040E000510560F7FA01EE52FF4F0C94842E853B88
:1040F00029F781E080933404E1CF823609F07DC056
:10410000C0923404DBCF8093330480933204D09286
:104110003404D4CF9C0133273093310420933004EE
:1041200090913204982790933204E0923404C6CFE1
:10413000382F22274091300450913104242B352B05
:104140003093310420933004909132049827909357
:104150003204F09234042536310508F4AFCF61E023
:1041600070E08CEC0E94B81D81E00E94991D0E94B5
:10417000D51D43C020912E0430912F04F901E65340
:10418000FC4F808390913204982790933204C901A8
:10419000019690932F0480932E0420913004309147
:1041A00031048217930708F489CF0093340486CF33
:1041B0008091320482130BC060912E0470912F0401
:1041C0004AEC53E0809133040E94DC1D0DC062E094
:1041D00070E08BEC0E94B81D809133040E94991D01
:1041E00080916A050E94991DFE01812F11928A9586
:1041F000E9F710922F0410922E04109234045ECF2F
:10420000CDB7DEB7E8E00C94732E81E080936B05A8
:1042100080916B05882349F082EE95E00E94B42BD3
:10422000892BB1F30E944C20F3CF0895AAE2B0E0AD
:10423000ECE1F1E20C94552E0E94A8286B017C0160
:1042400081E00E94B00A82EE95E00E94B42B892B97
:1042500029F082EE95E00E94E12BF5CF4398299852
:1042600011E072E6B72EE9E2AE2E03E00E94A82824
:104270006C197D098E099F09693C710581059105BD
:10428000F0F11123E1F10E94A8286B017C0185B1B6
:10429000846285B980ED97E00E94B607B982E6E7AF
:1042A000F5E0DE0112968A2D01900D928A95E1F7D4
:1042B0006AE2CE0101960E940D0C85B18B7D85B915
:1042C00080E090E00E94B607009373050E948B0B7C
:1042D00062E370E080E090E00E94D728809173054F
:1042E000843061F4009373058FE70E94A9090E944E
:1042F000BC0911E0823419F410E001C011E087E03C
:104300000E94CD29892BB1F411E014C0439A299A57
:1043100085B1846285B982EE95E00E94E12B8D30F3
:104320009105C1F074F40A97A9F04398299885B1D2
:104330008B7D85B982EE95E00E94B42B892B31F7F5
:1043400095CF8332910579F08234910571F70E94FF
:104350000521EBCF62EB71E082EE95E00E948E2AA0
:104360000E946F1DE2CF0E94F815DFCF8F929F92BF
:10437000AF92BF92CF92DF92EF92FF921F93CF93B3
:10438000DF9387E00E94CD29892B09F089C068EC72
:1043900070E080E090E00E94D72880E090E00E94EA
:1043A000B6070E94A8284B015C016B017C0180ECE0
:1043B000C80E82E1D81EE11CF11C0E94A8286C15D1
:1043C0007D058E059F0530F487E00E94CD29892B5D
:1043D000A1F364C087E00E94CD29892B09F05EC05B
:1043E00080ED97E00E94B6070E94A8286B017C012F
:1043F000D0E0C1E088E4880E86E2981EA11CB11CC2
:1044000011E087E00E94CD29892B21F58C149D04B1
:10441000AE04BF0430F480ED97E00E94B607D1E00F
:10442000F0CF0E94A8286C197D098E099F09693C6C
:1044300071058105910528F30E94A8286B017C0174
:10444000C12719F080ED97E002C080E090E00E9463
:10445000B607D7CF80E090E00E94B607DD23B9F021
:104460008091D30590E0019665E070E00E94F82D00
:104470008093D3050E944F0D0E94CF130E946F0DB1
:1044800064EF71E080E090E00E94D72809C080E0EE
:104490000E94DF060E94E7110E94660D0E9416210D
:1044A000DF91CF911F91FF90EF90DF90CF90BF9061
:1044B000AF909F908F900895CF92DF92EF92FF92EE
:1044C00080E00E940D080E94E40761E081E10E9403
:1044D000612961E08DE00E94612961E089E00E942C
:1044E000612961E08AE00E94612960E087E00E9422
:1044F000612960E088E00E94612961E088E00E9413
:104500009A290E949F0740E052EC61E070E082EE41
:1045100095E00E94FC2C0E94CF130E946F0D0E9418
:10452000B4138FEF8093AA040E94F90778940E9435
:10453000A8286B017C018091AA048F3F59F40E9446
:10454000A8286C197D098E099F09603D7740810577
:10455000910588F380ED97E00E94B60761E087E05F
:104560000E949A29439A299A82EE95E00E94B42BE0
:10457000892B29F082EE95E00E94E12BF5CF6DEFBB
:1045800072E082EE95E00E946F2A80E893E00E943C
:10459000620C64E173E082EE95E00E946F2A4AE0CB
:1045A00050E063E070E082EE95E00E943F2B62E312
:1045B00070E080E090E00E94D72882EE95E00E94B3
:1045C000B42B04970CF182EE95E00E94E12B82342B
:1045D0009105D1F482EE95E00E94E12B8E34910595
:1045E00099F482EE95E00E94E12B8434910561F408
:1045F00082EE95E00E94E12B819731F480E090E01B
:104600000E94B6070E9416214091770550917805C7
:104610006091790570917A05DB01CA010197A109C2
:10462000B1090497A105B10568F44093A90443308A
:1046300029F440EA56E861E070E004C040E052EC42
:1046400061E070E082EE95E00E94FC2C0E94B621B1
:104650004398299880E090E00E94B6070E94B41326
:104660001092C5048091BF0583FF11C080918B0516
:10467000882351F080919205882331F0809199052B
:10468000882311F087E001C085E08093C50480E0B5
:104690000E94B00A8091C6040E94E4090E948B0B1C
:1046A00010923F0410923E0410923D04F12C809130
:1046B000D4058F15B0F062E370E080E090E00E94D6
:1046C000D72880ED97E00E94B60762E370E080E0B3
:1046D00090E00E94D72880E090E00E94B607F39413
:1046E000E6CF80919E0584FF08C0982F987181E0E5
:1046F000983109F080E00E94A3118FE00E940D081C
:10470000FF90EF90DF90CF900895EF92FF920F937C
:104710001F93CF93DF938C016EE770E082EE95E0FC
:104720000E945906E801F12CF0E2EF2E8E018881FB
:104730008D57823048F46DE770E082EE95E00E947C
:10474000590688818E2588832196F801608182EE42
:1047500095E00E940E2CF394F9E0FF12E7CF6EE78C
:1047600070E082EE95E00E945906CDB7DEB7E6E034
:104770000C94752EA9E0B0E0E0ECF3E20C945D2E11
:104780009091C70491110EC09EEF99838A836B8329
:1047900050E0559547954C832D83198618861F82C6
:1047A0001E822EC04091CC04842F90E0B4E09595F9
:1047B0008795BA95E1F7242F2F7030E08217930781
:1047C00019F18DEF89831B82FE01349650E0842F0E
:1047D00090E0A4E095958795AA95E1F7242F2F7096
:1047E00030E08217930749F0DC01A353BB4F8C9153
:1047F0008193405F5F5F563051F74093CC045A83FA
:10480000CE0101960E9485238091C70490E0019615
:1048100066E070E00E94F82D8093C7042996E2E0DC
:104820000C94792EA0E0B0E0E8E1F4E20C94562E6E
:104830006C016EE770E082EE95E00E9459068601F9
:10484000E12CF12CC0E0D0E030E2B32EF801608121
:1048500083E8860F823078F46DE770E082EE95E0B1
:104860000E945906F80160816B2570E082EE95E0A8
:104870000E94590604C082EE95E00E940E2CE114BD
:10488000F10459F0F80180819E01280F311DC90102
:10489000C92FDD27C80FD91FDD273FEFE31AF30A21
:1048A00089E0E816F10459F028E0E216F10421F459
:1048B0008C2F8095F60180870F5F1F4FC7CFCDB734
:1048C000DEB7E9E00C94722EA9E0B0E0EAE6F4E28B
:1048D0000C945D2EE82F362F8091C70490E001964E
:1048E00064E270E00E94F82D8093C70458E9598370
:1048F00050E15A83813089F048F08230B9F083303A
:10490000D9F48B8381EF8C833D8319C085E08B8341
:1049100081EF8C832F5F2D8312C08B8381EF8C837B
:1049200084E6489FA00111245D8309C084E08B8345
:1049300081EF8C83ED8303C00E94E01104C0CE019F
:1049400001960E9412242996E2E00C94792EA2E0AE
:10495000B0E0EDEAF4E20C94522E182F762E2A8362
:1049600049830E94B4286B017C018091DD04809012
:10497000C8049090C904A090CA04B090CB042A81C6
:1049800049818823C1F0D701C60188199909AA096C
:10499000BB094C015D0191EE89169EE29906A104C6
:1049A000B10420F1241708F4422F202F672D812F06
:1049B0000E94642413C0D701C60188199909AA0965
:1049C000BB094C015D0191E3891695E79906A104A5
:1049D000B10460F0672D812F0E94BA23C092C804F1
:1049E000D092C904E092CA04F092CB042296EDE082
:1049F0000C946E2EA2E2B0E0E0E0F5E20C94532EAF
:104A00008CE00E94CB0981110FC06CE173E082EE53
:104A100095E00E94A02A439A299A80E00E94B00A59
:104A20000E948B0B4398299882EE95E00E94B42B4C
:104A3000892B01F182EE95E00E94E12B9091A9046F
:104A4000992319F00E94E213EFCF40913E0450E009
:104A50009A012F5F3F4F2F71332760913F0470E021
:104A60002617370709F3FA01E75BFB4F8083209392
:104A70003E04DACF80917305843009F086C00E942D
:104A8000B428611571058105910549F06093B7045B
:104A90007093B8048093B9049093BA040CC081E079
:104AA00090E0A0E0B0E08093B7049093B804A093A6
:104AB000B904B093BA048091AD049091AE048160C2
:104AC0009093AE048093AD0483E0809373058FE7E9
:104AD0000E94A90909E614E00E94BC09F80181932B
:104AE0008F01F4E002371F07B9F72091720480911B
:104AF0006904982F922796FF3BC090E492279093E9
:104B00007204982F98739833F1F410E0212F30E05D
:104B100080916904877090E0821793074CF11F5FC2
:104B200020919E05812F90E0FC01E759FB4F24FF67
:104B300004C080810E94C211E9CF608182EE95E0BD
:104B40000E940E2CE3CF8F7399F480916A048093B6
:104B5000B60480916B048093B40480916C048093BC
:104B6000B30480916F0490E09093AC048093AB0405
:104B700080913D04813019F482E080933D0480915E
:104B80003D04833011F410923D040E94B4286B015F
:104B90007C018091AF049091B004A091B104B091D8
:104BA000B2040097A105B105C9F0A7019601281B21
:104BB000390B4A0B5B0BDA01C901883B9B40A1050D
:104BC000B10560F00E94FA098093B5041092AF0419
:104BD0001092B0041092B1041092B2048091BB0400
:104BE0009091BC04A091BD04B091BE044601570150
:104BF000881A990AAA0ABB0A86E795E00E94270844
:104C000086169706A806B90608F4AAC0C092BB0487
:104C1000D092BC04E092BD04F092BE040E945706FC
:104C20008091AA048830A0F08091BF059091C005C2
:104C3000A091C105B091C2056CE1B695A795979575
:104C400087956A95D1F7892B8A2B8B2B09F0AAC1FE
:104C50008091AA048F5F8093AA048091B7049091F9
:104C6000B804A091B904B091BA040097A105B105A8
:104C7000F1F0C81AD90AEA0AFB0A86E795E00E9411
:104C800027086C157D058E059F0508F00AC18091E7
:104C9000BF0584FD04C080ED97E00E94B607109226
:104CA000B7041092B8041092B9041092BA0490910B
:104CB0007204907C9093720450913E0480913F0462
:104CC00020913D04581709F409C1223009F006C1AA
:104CD000905890937204E0919E05E770F0E0E658DA
:104CE000FC4F6081693008F0E1C0615040E046133C
:104CF000DFC080933F0487E3840F90917204892B77
:104D0000809372044093400483E080933D0485B116
:104D1000846285B9809183059091C504911133C156
:104D20000E94AB0A8091C6040E94E409E0919E05AE
:104D3000E770F0E0E658FC4F608182E794E00E9463
:104D4000C60BE091C604EF5FE093C604E83109F4B6
:104D500026C1F0E0EA58FA4F8785882309F41FC17D
:104D60000E94350C813069F580919E05887149F16A
:104D70008091AD049091AE04880F991F9093AE047A
:104D80008093AD0483E0809373050E948B0B0E9497
:104D9000B4286093AF047093B0048093B1049093EF
:104DA000B204672B682B692B61F481E090E0A0E0EE
:104DB000B0E08093AF049093B004A093B104B0939B
:104DC000B20480919E0584FF1FC08091AD04909134
:104DD000AE048E7F0E945D09182F6091AB04809114
:104DE000B6040E94D813482F612F8091B50449A3BF
:104DF0000E94D8130091D405282F49A16091B304D3
:104E00008091B4040E94A72485B18B7D85B98091DF
:104E1000C3048130C1F018F08230B1F1D1C087E015
:104E20000E94CD29892B09F0CBC081E08093C30477
:104E30000E94A8286093BF047093C0048093C104AB
:104E40009093C204BDC087E00E94CD29892B31F523
:104E50000E94A828C090BF04D090C004E090C10474
:104E6000F090C2046C197D098E099F09693E734058
:104E70008105910508F4A4C082E08093C30480ED0D
:104E800097E00E94B6079CC087E00E94CD29892B3D
:104E900009F496C080E090E00E94B6071092C30427
:104EA0008FC080E090E00E94B60701CF68E01ECF7F
:104EB000851709F41ECF4F5F242F30E090E0F901F1
:104EC000EE58FB4FDC01A75BBB4F7C917083F9016F
:104ED000E05CFB4F708301968F7109CF2430B1F4F1
:104EE0002091400481E494E0A3E7B4E0FC013E2F6C
:104EF000381B321718F431913D93F9CF87E3820FB5
:104F000090917204892B80937204FECE8091C30429
:104F1000823071F4916090937204439A299A53EC11
:104F2000E52E55E0F52E8E010F5F1F4FB80111C021
:104F30004398299880913D04811103C081E08093BA
:104F40003D0480913D04833051F784E080933D041B
:104F5000E6CFF70181917F0169A37AA30E94DA1558
:104F6000F801819391938F0169A17AA1F3EDEF1676
:104F7000F5E0FF0671F780919E0543E754E08770E6
:104F80000E94AC08C4CE882309F4CACE2091C40480
:104F900031E0320F3093C4042913C2CE0DC01092F9
:104FA000C604DECE8091AA04883011F4439A299A6F
:104FB00089E08093AA04D4CE1092C4048150B0CE6C
:104FC000A296ECE00C946F2E8230E8F4E82FF0E02B
:104FD000EE0FFF1FEB52FA4F71836083813041F077
:104FE000809169008C7F842B80936900E89A0895F2
:104FF00080916900440F551F440F551F837F842BF8
:1050000080936900E99A08951F920F920FB60F924C
:1050100011242F933F934F935F936F937F938F93BD
:105020009F93AF93BF93EF93FF938091D50590919A
:10503000D605892B29F0E091D505F091D605099583
:10504000FF91EF91BF91AF919F918F917F916F9160
:105050005F914F913F912F910F900FBE0F901F9036
:1050600018951F920F920FB60F9211242F933F9312
:105070004F935F936F937F938F939F93AF93BF9360
:10508000EF93FF938091D7059091D805892B29F054
:10509000E091D705F091D8050995FF91EF91BF9167
:1050A000AF919F918F917F916F915F914F913F91C0
:1050B0002F910F900FBE0F901F9018951F920F9277
:1050C0000FB60F9211242F933F938F939F93AF931B
:1050D000BF938091DA059091DB05A091DC05B0913A
:1050E000DD053091D90523E0230F2D3720F40196FB
:1050F000A11DB11D05C026E8230F0296A11DB11DFB
:105100002093D9058093DA059093DB05A093DC0505
:10511000B093DD058091DE059091DF05A091E0055B
:10512000B091E1050196A11DB11D8093DE0590931C
:10513000DF05A093E005B093E105BF91AF919F918A
:105140008F913F912F910F900FBE0F901F90189548
:105150002FB7F8946091DA057091DB058091DC053A
:105160009091DD052FBF08953FB7F8948091DE053B
:105170009091DF05A091E005B091E10526B5A89BCF
:1051800005C02F3F19F00196A11DB11D3FBF662735
:10519000782F892F9A2F620F711D811D911D42E07A
:1051A000660F771F881F991F4A95D1F70895CF92F0
:1051B000DF92EF92FF92CF93DF936B017C010E940D
:1051C000B428EB01C114D104E104F10479F00E9488
:1051D000B4286C1B7D0B683E7340A0F381E0C81AB5
:1051E000D108E108F108C851DC4FECCFDF91CF9135
:1051F000FF90EF90DF90CF900895789484B582600F
:1052000084BD84B5816084BD85B5826085BD85B56A
:10521000816085BDEEE6F0E0808181608083E1E819
:10522000F0E0108280818260808380818160808351
:10523000E0E8F0E0808181608083E1EBF0E0808154
:1052400084608083E0EBF0E0808181608083EAE726
:10525000F0E08081846080838081826080838081AF
:10526000816080838081806880831092C10008956E
:10527000833081F028F4813099F08230A1F00895D4
:105280008630A9F08730B9F08430D1F48091800065
:105290008F7D03C0809180008F7780938000089578
:1052A00084B58F7702C084B58F7D84BD08958091C9
:1052B000B0008F7703C08091B0008F7D8093B000E5
:1052C0000895CF93DF9390E0FC01ED50F44F2491CB
:1052D000FC01E95FF34F8491882349F190E0880F46
:1052E000991FFC01E15DF34FA591B4918B5D934F44
:1052F000FC01C591D4919FB7611108C0F8948C91BD
:10530000209582238C93888182230AC0623051F4D5
:10531000F8948C91322F309583238C938881822B43
:10532000888304C0F8948C91822B8C939FBFDF916B
:10533000CF910895A1E0B0E0E0EAF9E20C945B2E91
:10534000282F30E0F901E152F44F8491F901ED503A
:10535000F44F1491F901E95FF34F04910023C9F070
:10536000882321F069830E9438296981E02FF0E0C9
:10537000EE0FFF1FEB5DF34FA591B4919FB7F8942B
:105380008C91611103C01095812301C0812B8C93F6
:105390009FBF2196E4E00C94772ECF93DF93282FC4
:1053A00030E0F901E152F44F8491F901ED50F44FEE
:1053B000D491F901E95FF34FC491CC2391F08111AD
:1053C0000E943829EC2FF0E0EE0FFF1FE55EF34F4F
:1053D000A591B4912C912D2381E090E021F480E0FF
:1053E00002C080E090E0DF91CF9108958E3008F008
:1053F0008E50877020919D0190E4299F9001112487
:10540000822B80937C0080917A00806480937A0064
:1054100080917A0086FDFCCF809178002091790000
:1054200090E0922B0895A0E0B0E0E9E1FAE20C945C
:10543000572E6C017A01EB01E60EF71E00E010E03A
:10544000CE15DF0561F06991D601ED91FC910190D7
:10545000F081E02DC6010995080F191FF1CFC80191
:10546000CDB7DEB7E8E00C94732E6115710589F0B5
:10547000DB010D900020E9F7AD0141505109461BB9
:10548000570BDC01ED91FC910280F381E02D099531
:10549000089580E090E00895EF92FF920F931F939C
:1054A000CF93DF938C01FB01C0E0D0E064917F01DA
:1054B0008FEFE81AF80A662361F0D801ED91FC91AC
:1054C0000190F081E02DC8010995C80FD91FF7019F
:1054D000EDCFCE01CDB7DEB7E6E00C94752E0E947D
:1054E000352A0895DC01ED91FC910190F081E02DC9
:1054F000099508950F931F93CF93DF93EC016DE00F
:105500000E94722A8C016AE0CE010E94722A800FEA
:10551000911FDF91CF911F910F9108950F931F93CA
:10552000CF93DF93EC010E944C2A8C01CE010E94A4
:105530007A2A800F911FDF91CF911F910F910895CB
:105540000F931F93CF93DF93EC010E94352A8C01B8
:10555000CE010E947A2A800F911FDF91CF911F9177
:105560000F9108950F931F93CF93DF93EC010E9447
:10557000722A8C01CE010E947A2A800F911FDF913E
:10558000CF911F910F910895A1E2B0E0EAECFAE209
:105590000C94532E7C01C42EE52FCB01D22E19A2E0
:1055A00021E02D1510F02AE0D22E8E010F5D1F4F45
:1055B0008D2C912CA12CB12C6C2D7E2FA50194014A
:1055C0000E940C2E8C2DD29E80191124015011099D
:1055D0008A3010F4805D01C0895CF8018083211558
:1055E00031054105510521F0C22EE32FCA01E4CF58
:1055F000B801C7010E94352AA196ECE00C946F2EE9
:10560000A0E0B0E0E6E0FBE20C94572EEC016A016A
:105610007B012115310541F4E881F9810190F08188
:10562000E02D642F09951DC02A303105A9F477FFBC
:1056300012C06DE20E94722A8C0144275527BA01DC
:105640004C195D096E097F092AE0CE010E94C42A27
:10565000800F911F06C02AE0B701A601CE010E946B
:10566000C42ACDB7DEB7E8E00C94732E9A01AB01E3
:10567000662757FD6095762F0E94002B08950F93A3
:105680001F93CF93DF93EC019A01AB01662757FD7F
:105690006095762F0E94002B8C01CE010E947A2A01
:1056A000800F911FDF91CF911F910F9108952115C8
:1056B000310549F4DC01ED91FC910190F081E02D80
:1056C000642F099508950E94C42A08959A01462FCF
:1056D00050E060E070E00E94572B08959A01AB0102
:1056E00060E070E00E94572B08950F931F93CF93B3
:1056F000DF93EC010E94572B8C01CE010E947A2A85
:10570000800F911FDF91CF911F910F9108950F93FB
:105710001F93CF93DF93EC019A01AB0160E070E03F
:105720000E94572B8C01CE010E947A2A800F911F74
:10573000DF91CF911F910F9108950F931F93CF93F6
:10574000DF93EC019A01462F50E060E070E00E9488
:10575000572B8C01CE010E947A2A800F911FDF9176
:10576000CF911F910F910895FC0124853585F90192
:10577000E05CFF4F80819181F901EE5BFF4F20815A
:105780003181821B930B8F7399270895FC018485C7
:105790009585FC01E05CFF4F40815181FC01EE5B8F
:1057A000FF4F208131814217530741F00190F08172
:1057B000E02DE80FF91F808190E008958FEF9FEFB3
:1057C0000895FC0184859585FC01E05CFF4F4081D4
:1057D0005181FC01EE5BFF4F20813181421753075D
:1057E00079F0A081B181A80FB91F8C9120813181FE
:1057F0002F5F3F4F2F7333273183208390E008952D
:105800008FEF9FEF0895FC0181A1882329F0A489DF
:10581000B5898C9186FFFBCF11A20895CF93DF93BA
:10582000FC0126853785D901A05CBF4F8D919C91E5
:10583000119701968F739927E901CE5BDF4F48815D
:10584000598184179507D9F30D90BC91A02DA20F13
:10585000B31F6C93A685B785A05CBF4F11969C9330
:105860008E93A689B7892C9181E090E0078C02C0C5
:10587000880F991F0A94E2F7282B2C9381E081A3CB
:105880000488F589E02D80818064808381E090E048
:10589000DF91CF91089508951F920F920FB60F9246
:1058A00011242F933F934F938F939F93EF93FF93E5
:1058B0008091C00082FD1CC04091C6008091880686
:1058C0009091890601968F73992720918A063091CD
:1058D0008B068217930771F0E0918806F091890694
:1058E000E85BF94F4083909389068093880602C055
:1058F0008091C600FF91EF919F918F914F913F91C1
:105900002F910F900FBE0F901F90189582EE95E08B
:105910000E94B42B892B11F00E944B2C08951F92EA
:105920000F920FB60F9211242F933F938F939F9353
:10593000EF93FF93209144063091450680914606EF
:10594000909147062817390731F48091C1008F7D67
:105950008093C10014C0E0914606F0914706EC5FC9
:10596000F94F2081809146069091470601968F73EA
:10597000992790934706809346062093C600FF918F
:10598000EF919F918F913F912F910F900FBE0F90AC
:105990001F901895A0E0B0E0E0EDFCE20C94532ECF
:1059A000FC011382128288EE93E0A0E0B0E08483D1
:1059B0009583A683B7838CEB93E09183808375876F
:1059C000648757874687318B208B138B028BF58A30
:1059D000E48AD78AC68AB18EA08E938E828E8F85F6
:1059E000848F8889858F8989868F8A89878F8B891B
:1059F00080A3ECE00C946F2ECF92DF92EF92FF9297
:105A0000CF93DF93EC016A017B01411581EE5807CA
:105A100061057105F9F0EC89FD8981E090E008A04D
:105A200002C0880F991F0A94E2F7808360E079E052
:105A30008DE390E0A70196010E940C2E21503109C0
:105A4000410951095695479537952795211580E1CC
:105A5000380798F0EC89FD89108260E874E88EE1DF
:105A600090E0A70196010E940C2E215031094109B6
:105A700051095695479537952795E889F9893083D7
:105A8000EA89FB89208319A2EE89FF89408181E0A0
:105A900090E09C010C8C02C0220F331F0A94E2F7A5
:105AA000422B4083EE89FF8940819C010D8C02C00E
:105AB000220F331F0A94E2F7422B4083EE89FF89BD
:105AC00040819C010E8C02C0220F331F0A94E2F722
:105AD000422B4083EE89FF8920810F8C02C0880F02
:105AE000991F0A94E2F7809582238083DF91CF91FA
:105AF000FF90EF90DF90CF9008958F929F92AF929A
:105B0000BF92CF92DF92EF92FF920F931F9381E0AB
:105B10008F9385E08F9387E08F9383E08F9384E06A
:105B20008F93E6EC8E2E912CF2ECAF2EB12CA1ECE3
:105B3000CA2ED12CB0ECEB2EF12C04EC10E025ECAD
:105B400030E044E056E068E476E082EE95E00E94C2
:105B5000CA2C0F900F900F900F900F901F910F91E4
:105B6000FF90EF90DF90CF90BF90AF909F908F907D
:105B700008950E94FD280E945C22C6E8DCE20E9493
:105B8000FA242097E1F30E94862CF9CFA29FB0015E
:105B9000B39FC001A39F700D811D1124911DB29F61
:105BA000700D811D1124911D08950E94C62DA59F81
:105BB000900DB49F900DA49F800D911D1124089508
:105BC000B7FF0C94D52D0E94D52D821B930B089501
:105BD000DB018F939F930E94D52DBF91AF91A29F20
:105BE000800D911DA39F900DB29F900D11240895DB
:105BF00097FB072E16F4009407D077FD09D00E947A
:105C00008A2E07FC05D03EF4909581959F4F08950C
:105C1000709561957F4F0895A1E21A2EAA1BBB1BB8
:105C2000FD010DC0AA1FBB1FEE1FFF1FA217B30768
:105C3000E407F50720F0A21BB30BE40BF50B661F7E
:105C4000771F881F991F1A9469F760957095809542
:105C500090959B01AC01BD01CF010895052E97FBE6
:105C60001EF400940E94452E57FD07D00E940C2E72
:105C700007FC03D04EF40C94452E5095409530957A
:105C800021953F4F4F4F5F4F0895909580957095A8
:105C900061957F4F8F4F9F4F08952F923F924F9264
:105CA0005F926F927F928F929F92AF92BF92CF92AC
:105CB000DF92EF92FF920F931F93CF93DF93CDB7B5
:105CC000DEB7CA1BDB0B0FB6F894DEBF0FBECDBF2D
:105CD00009942A88398848885F846E847D848C84FE
:105CE0009B84AA84B984C884DF80EE80FD800C8107
:105CF0001B81AA81B981CE0FD11D0FB6F894DEBFEA
:105D00000FBECDBFED010895EE0FFF1F0590F4917A
:105D1000E02D0994AA1BBB1B51E107C0AA1FBB1FA2
:105D2000A617B70710F0A61BB70B881F991F5A9527
:105D3000A9F780959095BC01CD0108958F929F920F
:105D4000AF92BF92CF92DF92EF92FF92CF93DF9309
:105D5000EC01688179818A819B81611571058105DA
:105D6000910521F464E279ED8BE597E02DE133EFC5
:105D700041E050E00E942E2E49015A019B01AC01E6
:105D8000A7EAB1E40E94D52D6B017C01ACEEB4EF23
:105D9000A50194010E94E32DC60ED71EE81EF91E30
:105DA000F7FE06C081E0C81AD108E10880E8F80AC9
:105DB000C882D982EA82FB82C701B6019F77DF9150
:105DC000CF91FF90EF90DF90CF90BF90AF909F90DA
:105DD0008F9008950E949E2E089586E091E00E9483
:105DE0009E2E089560930601709307018093080129
:105DF0009093090108952F923F925F926F927F9244
:105E00008F929F92AF92BF92CF92DF92EF92FF92CA
:105E10000F931F93CF93DF938B01EA0161157105F7
:105E200021F0DB018C9311969C93209739F09E0111
:105E3000225031092332310508F0D8C07C016701B6
:105E4000BFEFCB1ADB0A5601F7016080862D90E088
:105E50000E942D30892B11F07601F1CFFDE26F12F7
:105E60000AC0570182E0A80EB11CD70111966C90B0
:105E7000772473940BC0BBE26B1207C05701E2E0BA
:105E8000AE0EB11CD70111966C90712CCE018F7E95
:105E9000892B89F4B0E36B1237C0F50180818F7DC7
:105EA0008835D1F46180F2E0AF0EB11C872D82609D
:105EB000782EC0E1D0E0CA30D10551F1C031D10512
:105EC00021F0C830D10599F409C0CC24CA94DC2C47
:105ED000EC2CAFE0FA2E22C0209769F7C8E0D0E0A2
:105EE000CC24CA94DC2CEC2CFFE1FF2E17C06FEF02
:105EF0007FEFCB019E01442737FD4095542F0E9430
:105F00000C2E69017A010AC02097A9F6CAE0D0E0F8
:105F1000E9E9CE2EDC2CEC2CE9E1FE2EF50160E067
:105F200020E030E0A9014E01AA2497FCA094BA2CED
:105F30001F0170ED572E560CA9E0A51570F48FEBDC
:105F4000860D8A3118F499EC592E06C08FE9860D1A
:105F50008A3148F589EA582E560C852D90E08C1729
:105F60009D070CF56F3FD9F0C216D306E406F5067F
:105F700098F0C501B4010E94E82D9B01AC01852D6C
:105F800090E0A0E0B0E0280F391F4A1F5B1F2817E0
:105F900039074A075B0710F46FEF01C061E03196E3
:105FA000D1016C90C5CF0115110551F0662311F098
:105FB000319703C071FE04C03297D801ED93FC9372
:105FC00070FE07C050954095309521953F4F4F4F3B
:105FD0005F4F67FF10C082E290E090938D06809340
:105FE0008C066FEF7FEF8FEF9FEF07C060E070E0F0
:105FF00080E090E002C0B901CA01DF91CF911F910A
:106000000F91FF90EF90DF90CF90BF90AF909F9057
:106010008F907F906F905F903F902F900895FC013C
:1060200088279927E89421912032E9F3293010F04C
:106030002E30C8F32B3241F02D3239F4689404C06D
:106040000E946130820F911D219120532A30C0F3AC
:106050001EF4909581959F4F0895911150C0803204
:1060600019F089508550D0F7089548EC53E00E940C
:106070003A300895FA01A191B081009719F4109770
:10608000E1F0CD01DC01CD010D90002011F4C00143
:1060900013C0FB012191222319F02015D9F7F3CF6A
:1060A000FB012191201519F41E92119606C022239E
:1060B000C1F70D900020A1F7D001FA01A193B083A0
:1060C00008957AE0979F902D879F802D910D112440
:1060D0000895F999FECF92BD81BDF89A992780B5B0
:1060E0000895262FF999FECF1FBA92BD81BD20BD1C
:1060F0000FB6F894FA9AF99A0FBE01960895992767
:0861000088270895F894FFCFF1
:1061080000008E06200001000000FF0002000200CF
:106118000200020002000200020002000200020067
:1061280002000200020002000200028025000005B1
:10613800400AA1204EA50020244EA52C2330C012D1
:1061480000001A400AA1204EA5001B1E27522C232E
:10615800308025000005400AA1204EA50020244ECD
:10616800A52C2330004B000006400AD0009D4900B2
:106178007B289D492C233000E1000005400A450199
:10618800D7DC03B81E0EBF00232E48E801008A4062
:106198000A6001555502AD1E20000023C80154585D
:1061A8002074696D656F75742100596573004E6FB1
:1061B800002C00386368004E2F41002C205B005DE6
:1061C8002028002900486F70206368616E6E656C36
:1061D800200020402000456E746572696E6720615A
:1061E80064617074697665206368616E6E656C20A1
:1061F80073656C656374696F6E2C207069636B6975
:106208006E673A007363616E6E6572206D6F6465C8
:10621800004E4F5420454E41424C45440053656E54
:1062280064696E672073657474696E677320746F30
:106238002052580A00526573657474696E6720733A
:10624800657474696E6773206F6E2052580A004136
:10625800626F727465642065646974730A00696E9C
:1062680076616C69642073656C656374696F6E0030
:106278000D0A496E76616C696420696E70757420C8
:106288002D20646973636172646564210700536536
:106298007474696E677320736176656420746F2007
:1062A800454550524F4D0A005265766572746564D3
:1062B8002073657474696E67732066726F6D20450C
:1062C8004550524F4D0A004C6F6164656420666109
:1062D80063746F72792064656661756C74730A0003
:1062E8004B657920616E64206368616E6E656C73BE
:1062F8002072616E646F6D697A65640A004F70651B
:106308006E4C52536E6720545820737461727469CE
:106318006E672000206F6E20485720006D6F6475EF
:106328006C65206C6F636B65643F00342B340038F8
:1063380000382B340031320031322B340031360032
:1063480050504D0052535349005344410053434C5D
:1063580000525844005458440041494E004C4245AC
:1063680045500053504B54524D005342555300531F
:10637800554D44004C4C494E440000070B0C10117D
:106388001500B7012B032F033103350338033D03F1
:10639800B7014003440349034D035103550359030F
:1063A8005D0363036A036F0374038D028D028D021C
:1063B8008D02160A13223129000000000E2C132A20
:0863C800B42BE12BC62B032CC2
:107E00000F92CDB7DEB7112484B714BE81FFF1D035
:107E100082E08093C00088E18093C10086E0809377
:107E2000C20080E18093C4008EE0CDD088249924E4
:107E3000CC24C394F5E0DF2EE1E1EE2E73E0F72EC3
:107E4000B6D0082F813479F4B2D08983C2D0898129
:107E5000823811F481E005C0813811F485E001C059
:107E600083E09ED09AC0823411F484E103C085344B
:107E700019F485E0B6D091C0853561F498D0082F0B
:107E800010E095D090E0982E8824802A912A880CC2
:107E9000991C82C0863521F484E0A3D080E0E1CF34
:107EA000843609F04CC083D082D0A82E80D0B82E62
:107EB00000E011E07CD0F80181938F01AE16D1F77C
:107EC00088D0FB2DF53489F4E0E0F1E00BC0F9999E
:107ED000FECF92BC81BC0894811C911C819180BD15
:107EE000FA9AF99AEA1598F358C08B2D863409F05E
:107EF00054C0F401F7BEE89507B600FCFDCFF401CD
:107F0000A0E0B1E02C9130E011968C91119790E0B7
:107F1000982F8827822B932B12960C01C7BEE895C9
:107F20001124329681E0A038B80761F7F401D7BE7A
:107F3000E89507B600FCFDCFE7BEE8952EC0843774
:107F4000F1F435D034D0182F32D0B82E42D0FB2DDA
:107F5000F63421F4F40105914F010CC0FB2DF534EA
:107F600049F4F999FECF92BC81BC0894811C911C04
:107F7000F89A00B5802F14D0115049F70EC08537FC
:107F800039F427D08EE10CD085E90AD08FE069CF93
:107F9000813511F488E017D01CD080E101D050CF9A
:107FA0009091C00095FFFCCF8093C600089580910A
:107FB000C00087FFFCCF8091C00084FD01C0A89560
:107FC0008091C6000895E0E6F0E098E19083808318
:107FD0000895EDDF803219F088E0F5DFFFCF84E10E
:107FE000DFCF1F93182FE3DF1150E9F7F2DF1F9166
:0E7FF0000895282E80E0E7DFEE27FF27099492
:027FFE0001057B
:0400000300007E007B
:00000001FF
